:100000000C9446000C9465000C9465000C946500FB
:100010000C9465000C94A9000C940B010C946D01D8
:100020000C94CF010C946E000C9465000C94650048
:100030000C9465000C9465000C9465000C946500AC
:100040000C9465000C9465000C9465000C9465009C
:100050000C9465000C9465000C9465000C9465008C
:100060000C9465000C9465000C9465000C9465007C
:100070000C9465000C9465000C9465000C9465006C
:100080000C9465000C94B7050C94650011241FBEF8
:10009000CFEFD0E1DEBFCDBF12E0A0E0B1E0E6E2FD
:1000A000F6E100E00BBF02C007900D92A031B1074E
:1000B000D9F713E0A0E1B2E001C01D92AA34B10764
:1000C000E1F70E9433030C94110B0C9400008BE0B9
:1000D00085BD89EF83BD80E887BF08951F920F9289
:1000E0000FB60F9211248F939F93AF93BF9380917C
:1000F000100290911102A0911202B0911302019688
:10010000A11DB11D8093100290931102A0931202C1
:10011000B0931302BF91AF919F918F910F900FBE3B
:100120000F901F901895F89489B78F7089BF85E557
:100130008ABF80EF88BF89B7806F89BF789412B873
:100140008FEF84BB08958FEF84BB12B883B985BB52
:1001500008951F920F920FB60F920BB60F921124B3
:10016000EF92FF920F931F932F933F934F935F93C1
:100170006F937F938F939F93AF93BF93EF93FF936F
:1001800085B3809585BB60911002709111028091BA
:10019000120290911302E0901602F09017027093F1
:1001A000170260931602E6E1F2E032972081318176
:1001B0002F5F3F4F3183208300E010E06E197F09ED
:1001C000800B910B0E94CD089B01AC0160E070E0B8
:1001D00080E89FE30E94230860931802709319023D
:1001E00080931A0290931B02FF91EF91BF91AF9100
:1001F0009F918F917F916F915F914F913F912F913F
:100200001F910F91FF90EF900F900BBE0F900FBEBC
:100210000F901F9018951F920F920FB60F920BB66A
:100220000F921124EF92FF920F931F932F933F93FE
:100230004F935F936F937F938F939F93AF93BF93EE
:10024000EF93FF9385B3809585BB60911002709109
:1002500011028091120290911302E0901F02F0901F
:1002600020027093200260931F02EFE1F2E03297C8
:10027000208131812F5F3F4F3183208300E010E0E8
:100280006E197F09800B910B0E94CD089B01AC0178
:1002900060E070E080E89FE30E9423086093210201
:1002A000709322028093230290932402FF91EF9196
:1002B000BF91AF919F918F917F916F915F914F917E
:1002C0003F912F911F910F91FF90EF900F900BBED8
:1002D0000F900FBE0F901F9018951F920F920FB6A0
:1002E0000F920BB60F921124EF92FF920F931F9370
:1002F0002F933F934F935F936F937F938F939F932E
:10030000AF93BF93EF93FF9385B3809585BB6091C7
:100310001002709111028091120290911302E090EC
:100320002802F09029027093290260932802E8E2E3
:10033000F2E03297208131812F5F3F4F318320835C
:1003400000E010E06E197F09800B910B0E94CD0830
:100350009B01AC0160E070E080E89FE30E9423080D
:1003600060932A0270932B0280932C0290932D02AB
:10037000FF91EF91BF91AF919F918F917F916F917D
:100380005F914F913F912F911F910F91FF90EF90AF
:100390000F900BBE0F900FBE0F901F9018951F92DD
:1003A0000F920FB60F920BB60F921124EF92FF929D
:1003B0000F931F932F933F934F935F936F937F936D
:1003C0008F939F93AF93BF93EF93FF9385B38095E4
:1003D00085BB609110027091110280911202909180
:1003E0001302E0903102F090320270933202609377
:1003F0003102E1E3F2E03297208131812F5F3F4FFC
:100400003183208300E010E06E197F09800B910B8F
:100410000E94CD089B01AC0160E070E080E89FE3A2
:100420000E94230860933302709334028093350254
:1004300090933602FF91EF91BF91AF919F918F9171
:100440007F916F915F914F913F912F911F910F91EC
:10045000FF90EF900F900BBE0F900FBE0F901F906C
:100460001895BF92CF92DF92EF92FF920F931F9356
:10047000CF93DF93B62EEC01FC01E85CFD4F808149
:100480008F5F8083843009F092C0F894209110022D
:1004900030911102409112025091130278948E0112
:1004A00093E0000F111F9A95E1F70C0F1D1F0C5ED2
:1004B0001D4FF80182819381A0E0B0E069017A01CB
:1004C000C81AD90AEA0AFB0A338322838081918100
:1004D000019691838083C701B6010E94CD089B01DC
:1004E000AC0160E070E080E89FE30E942308F8011F
:1004F0006483758386839783FE01EC5FFE4FB08231
:10050000FE01E85CFD4F1082F80180858F5F8087D7
:1005100085EA80933C02C0923D02CD2CDE2CEF2C6C
:10052000FF24C0923E02C130D105C9F0C130D105CF
:1005300030F0C230D10511F12397C9F52FC0809159
:100540001C028823A1F181E080933F0244E06CE328
:1005500072E089E00E94C80710921C0225C08091B9
:100560002502882321F110923F0244E06CE372E0FF
:1005700089E00E94C8071092250216C080912E02C1
:100580008823A9F081E080933F0244E06CE372E0AD
:100590008AE00E94C80710922E0206C043E06CE376
:1005A00072E08FE00E94C80785B3809585BBDF911C
:1005B000CF911F910F91FF90EF90DF90CF90BF9060
:1005C0000895EF92FF920F931F93CF93DF9300E074
:1005D00011E0C0E0D0E021E0E22EF12C81B19E01DB
:1005E0002C5F3F4FB701022E02C0660F771F0A949F
:1005F000E2F790E06823792302C0759567952A9504
:10060000E2F7962FF8018081681759F4FE01EC5F3C
:10061000FE4F8081681729F070E0CE010E94310200
:1006200006C0F8019083FE01E85CFD4F1082219620
:100630000F5F1F4FC430D10589F6DF91CF911F9115
:100640000F91FF90EF90089543E06CE372E081E03A
:100650000E94C807882321F484E293E00E94610588
:10066000089508950895EF92FF920F931F93F894C1
:100670000E9482050E94670080E18093490360E048
:1006800070E080E090E00E94940560E070E080E01F
:1006900090E00E94A3008FEF84BB85BB92E3E92E1C
:1006A000F12C02E010E021E030E040E050E060E0BA
:1006B00070E081EE92E00E947003789482E3E82E6D
:1006C000F12C04E610E021E030E040E050E060E092
:1006D00070E082E393E00E9470030E946804FDCF03
:1006E000CF92DF92EF92FF920F931F93CF93DF93FE
:1006F000EC016B01A0E0B0E09A2FFD0184E0EE0F69
:10070000FF1F8A95E1F7EA0FFB1FEE5BFD4F878520
:10071000882329F09F5F1196AC30B10569F7692FE6
:1007200070E0FB01A4E0EE0FFF1FAA95E1F7E60FD2
:10073000F71FEE5BFD4FD183C083D382C282558306
:10074000448337832683E114F10411F4108A08C02E
:1007500082E3E816F10411F481E001C082E0808BAD
:10076000FB0134E0EE0FFF1F3A95E1F7E60FF71FAC
:10077000EE5BFD4FA089B0E0A25FBC4F8C91982F3B
:100780009E0D96878F5F8C931187008781E0878706
:10079000F894209110023091110240911202509170
:1007A0001302C801A0E0B0E0820F931FA41FB51F81
:1007B000FB0124E0EE0FFF1F2A95E1F7E60FF71F7C
:1007C000EE5BFD4F82879387A487B5877894DF918E
:1007D000CF911F910F91FF90EF90DF90CF900895F0
:1007E000CF92DF92EF92FF920F931F93CF93DF93FD
:1007F000DC01EB01690120E030E0622FF90174E0D7
:10080000EE0FFF1F7A95E1F7E20FF31FEE5BFD4F4E
:100810008785882331F06F5F2F5F3F4F2C30310584
:1008200061F7262F30E0F90164E0EE0FFF1F6A95B3
:10083000E1F7E20FF31FEE5BFD4FB183A083D3839B
:10084000C28355834483D782C682E114F10411F434
:10085000108A08C082E3E816F10411F481E001C0B7
:1008600082E0808BB90194E0660F771F9A95E1F7DB
:10087000620F731F6E5B7D4FEB01E889F0E0E25F72
:10088000FC4F8081982F9E0D9E878F5F80831987F4
:10089000088781E08F8720911002309111024091EA
:1008A000120250911302C801A0E0B0E0820F931F22
:1008B000A41FB51FFB0182879387A487B587DF91AB
:1008C000CF911F910F91FF90EF90DF90CF900895FF
:1008D000EF92FF920F931F93CF93DF93F894E090E2
:1008E0001002F090110200911202109113027894FC
:1008F00010921103809114038F5F809314038091F1
:100900001403883C49F48091130386958093120365
:1009100010921303109214034FEF5FEF20E030E0CA
:10092000F901A4E0EE0FFF1FAA95E1F7E20FF31F14
:10093000EE5BFD4F8785882399F0809111038F5FCF
:100940008093110382859385A485B585E816F90601
:100950000A071B0728F08685851710F45685422F55
:100960002F5F3F4F2C303105D9F64F3FB9F18091C1
:1009700013038F5F80931303842F992787FD90952E
:10098000EC01E4E0CC0FDD1FEA95E1F7C80FD91FB9
:10099000CE5BDD4FE881F9816C817D818A819B810D
:1009A00009958E819F81892B49F41F86E889F0E0A3
:1009B000E25FFC4F80818150808310C02A853B8597
:1009C0004C855D8588859985A0E0B0E0820F931FF6
:1009D000A41FB51F8A879B87AC87BD8781E0DF9105
:1009E000CF911F910F91FF90EF9008959C01DB0133
:1009F00060E070E0FB0144E0EE0FFF1F4A95E1F775
:100A0000E60FF71FEE5BFD4F808191818217930700
:100A100019F58785882301F1F8942091100230910F
:100A200011024091120250911302CD01A0E0B0E0FA
:100A3000820F931FA41FB51FFB0124E0EE0FFF1FC1
:100A40002A95E1F7E60FF71FEE5BFD4F828793874C
:100A5000A487B587789408956F5F7F4F6C307105D8
:100A600049F60895AC0120E030E0F901A4E0EE0F72
:100A7000FF1FAA95E1F7E20FF31FEE5BFD4F8081A8
:100A8000918184179507B9F487858823A1F0209177
:100A90001002309111024091120250911302CB01C9
:100AA000A0E0B0E0820F931FA41FB51F8287938739
:100AB000A487B58708952F5F3F4F2C303105A9F6E5
:100AC0000895AC0120E030E0F901B4E0EE0FFF1F23
:100AD000BA95E1F7E20FF31FEE5BFD4F8081918144
:100AE0008417950749F41786E089F0E0E25FFC4F30
:100AF00080818150808308952F5F3F4F2C303105D6
:100B000019F7089580E090E0FC0124E0EE0FFF1F4C
:100B10002A95E1F7E80FF91FEE5BFD4F1786019666
:100B20008C30910589F7089580914903880F816081
:100B30008093720080E480937000E1E7F0E08081B0
:100B40008C7F80832FEF2093730085EC809374005B
:100B500081E090E09093180380931703109216039E
:100B60002093430310922D0310922C0308951F929B
:100B70000F920FB60F920BB60F921124EF92FF92C5
:100B80000F931F932F933F934F935F936F937F9395
:100B90008F939F93AF93BF93EF93FF93809117032E
:100BA00090911803817C09F4CBC08091710090E092
:100BB000887F90708038910561F181389105ACF49F
:100BC0008836910509F48AC0893691052CF480365F
:100BD000910509F0B3C09AC08037910509F496C019
:100BE0008837910509F0AAC079C08039910589F04C
:100BF000813991052CF48838910509F09FC096C081
:100C00008839910509F492C0803A910509F096C09F
:100C100093C080911703909118038034910581F45B
:100C20008091730080931A038FEF8093430380E8D1
:100C300090E09093180380931703109216037CC0E2
:100C400080911703909118038038910509F074C0C2
:100C50009091160380911A039817A0F480911603BF
:100C6000E82FF0E090917300E75EFC4F92838F5F76
:100C7000809316039091430380917300892780939A
:100C800043035AC080911603803111F5809173009F
:100C900080932B039091430380912B03981719F0B5
:100CA00081E090E002C082E090E090932D03809379
:100CB0002C03EE24FF2400E010E020E030E040E0D0
:100CC00050E069E173E081E393E00E94F0032EC0FD
:100CD000809116038F5F809316032EC08091470387
:100CE0008F5F80934703809144038A3078F422E336
:100CF000E22EF12C02E310E020E030E040E050E092
:100D000060E070E08CE897E00E94F003809173004F
:100D10008093190310922D0310922C031092160346
:100D200085EC8093740080E490E07DC081E090E0E9
:100D3000909318038093170385ECD5C085E4D3C046
:100D40008091710090E0887F90708032910509F465
:100D50009CC08132910554F48031910599F088311D
:100D60009105D1F0089709F0B7C00CC08033910508
:100D700009F45EC08833910509F460C0889709F0D2
:100D8000ABC011C080912E038093730085E88093DF
:100D9000740088E090E047C01092150380912F0303
:100DA000809373003BC0809115038131D9F485E9AC
:100DB0008093740080E290E090931803809317036F
:100DC00010924403809145039091460301969093BD
:100DD00046038093450360E070E084E995E00E945B
:100DE000320583C09091150380912F03981750F01E
:100DF0008091400380937300809115038F5F8093EF
:100E000015030CC090911503E92FF0E0E25DFC4F53
:100E10008281809373009F5F9093150385E8809390
:100E2000740080E190E090931803809317035DC0F5
:100E3000809147038F5F809347032CC080914703C5
:100E40008F5F8093470360E070E084E995E00E9443
:100E50003205809144038A3080F492E3E92EF12C2C
:100E600002E310E020E030E040E050E060E070E0BD
:100E70008CE897E00E94F00306C088E290E090932F
:100E800018038093170385E82EC0809148038F5F75
:100E90008093480360E070E084E995E00E943205A9
:100EA000809144038A3080F482E3E82EF12C02E33F
:100EB00010E020E030E040E050E060E070E08CE8DE
:100EC00097E00E94F00306C088E290E09093180338
:100ED0008093170385E907C084E090E0909318039E
:100EE0008093170385E080937400FF91EF91BF9189
:100EF000AF919F918F917F916F915F914F913F91B2
:100F00002F911F910F91FF90EF900F900BBE0F90BC
:100F10000FBE0F901F901895EF92FF920F931F93A3
:100F20008091170390911803019771F042E3E42E2A
:100F3000F12C05E010E020E030E040E050E060E01F
:100F400070E08CE897E01DC01092150385EA80934D
:100F5000740082E090E090931803809317038091CF
:100F600044038F5F8093440332E3E32EF12C00E1CE
:100F700017E220E030E040E050E060E070E084E91B
:100F800095E00E9470031F910F91FF90EF900895DC
:100F9000EF92FF920F931F93582F80914403882361
:100FA00009F448C0809144038A3009F443C081E0C9
:100FB0003CC08FEF80934003DB0120E030E00DC0A8
:100FC0008C91F901E25DFC4F8283809140039D91F9
:100FD0008927809340032F5F3F4F241788F381E0D8
:100FE00080934403852F90E0880F991F80932E03F0
:100FF00040932F031092150385EA8093740082E0DA
:1010000090E0909318038093170352E3E52EF12CA0
:1010100005E010E020E030E040E050E060E070E00B
:1010200084E995E00E94700380E01F910F91FF908A
:10103000EF9008958091170390911803019709F498
:10104000B8CF82E0F2CFA8E1B0E0E9E2F8E00C949A
:10105000E20A69837A838B839C832D833E834F834B
:101060005887B9E0EB2EF12CEC0EFD1EB701CE0136
:1010700001960E946A0A8E010F5E1F4FB801CE01D1
:1010800005960E946A0A2985223008F47CC03989B5
:10109000323010F4B8017AC08A859A8989278A8704
:1010A000243011F0223031F4231709F06CC068E0CD
:1010B00071E06CC0343039F41D861E861F86188A94
:1010C0001C861B8604C0323021F484E08987B70176
:1010D0005DC02B853C858B899C89281B390B3C87FF
:1010E0002B87ED84FE840F851889AD88BE88CF8854
:1010F000D88CEA14FB040C051D0540F4EE0CFF1C13
:10110000001F111F215030403C872B8720E030E02A
:1011100040E050E080E090E0A0E0B0E46FE170E0FB
:10112000EA14FB040C051D0540F0282B392B4A2B33
:101130005B2BEA18FB080C091D09B695A795979536
:101140008795EE0CFF1C001F111F6150704041F786
:10115000DA01C9018F779070A070B070803491056A
:10116000A105B10561F427FD0AC0E114F1040105F0
:10117000110529F0205C3F4F4F4F5F4F20782D879E
:101180003E874F87588BBE01675F7F4FCB010E9420
:1011900095096896EAE00C94FE0AA8E0B0E0E3ED59
:1011A000F8E00C94E40A7B018C016115710581055E
:1011B000910519F482E0898360C083E089838EE120
:1011C000C82ED12CDC82CB82ED82FE820F83188761
:1011D000C801B7010E944609BC016150704077FF09
:1011E00039C0EE27FF27E61BF70B20E030E040E098
:1011F00050E081E090E0A0E0B0E00E2E04C0880F47
:10120000991FAA1FBB1F0A94D2F70197A109B10920
:101210008E219F21A023B1230097A105B10521F0C4
:1012200021E030E040E050E004C016950795F794C7
:10123000E794EA95D2F72E293F29402B512B2D8395
:101240003E834F8358878EE190E0861B970B9C83EB
:101250008B8313C06115710581F0062E04C0EE0C5E
:10126000FF1C001F111F0A94D2F7ED82FE820F832C
:101270001887C61AD70ADC82CB821A82CE01019661
:101280000E9495092896E8E00C94000BEF92FF92DB
:101290000F931F937B018C0180E0E81680E0F80635
:1012A00081E0080780E0180788F48FEFE816F10462
:1012B0000105110531F028F088E090E0A0E0B0E0F1
:1012C00017C080E090E0A0E0B0E012C080E0E81637
:1012D00080E0F80680E0080781E0180728F088E140
:1012E00090E0A0E0B0E004C080E190E0A0E0B0E0D9
:1012F00020E230E040E050E0281B390B4A0B5B0B4A
:1013000004C016950795F794E7948A95D2F7F701EC
:10131000E05FFE4F8081281B310941095109C90155
:101320001F910F91FF90EF900895DF92EF92FF923F
:101330000F931F93FC01E480F58006811781D18013
:101340008081823048F480E090E0A0E1B0E0E82ABB
:10135000F92A0A2B1B2BA5C0843009F49FC08230C8
:1013600021F4EE24FF24870105C0E114F1040105F6
:10137000110519F4E0E0F0E096C0628173819FEFFF
:10138000623879070CF05BC022E83FEF261B370B71
:101390002A3131052CF020E030E040E050E02AC056
:1013A000B801A701022E04C0769567955795479519
:1013B0000A94D2F781E090E0A0E0B0E004C0880F8A
:1013C000991FAA1FBB1F2A95D2F70197A109B1093E
:1013D0008E219F21A023B1230097A105B10521F003
:1013E00081E090E0A0E0B0E09A01AB01282B392B1E
:1013F0004A2B5B2BDA01C9018F779070A070B07017
:1014000080349105A105B10539F427FF09C0205C9E
:101410003F4F4F4F5F4F04C0215C3F4F4F4F5F4FD7
:10142000E0E0F0E02030A0E03A07A0E04A07A0E4C6
:101430005A0710F0E1E0F0E079018A0127C0603836
:10144000710564F5FB01E158FF4FD801C7018F77A3
:101450009070A070B07080349105A105B10539F489
:10146000E7FE0DC080E490E0A0E0B0E004C08FE3B0
:1014700090E0A0E0B0E0E80EF91E0A1F1B1F17FF66
:1014800005C016950795F794E794319687E0169571
:101490000795F794E7948A95D1F705C0EE24FF24C9
:1014A0008701EFEFF0E06E2F679566276795902F25
:1014B0009F77D794DD24D7948E2F8695492F462B7E
:1014C000582F5D29B701CA011F910F91FF90EF902E
:1014D000DF900895FC01DB01408151812281622F60
:1014E0006F7770E0221F2227221F9381892F880F98
:1014F000822B282F30E0991F9927991FFD01918396
:101500002115310581F5411551056105710511F46C
:1015100082E032C082E89FEFFD01938382839A01CB
:10152000AB0167E0220F331F441F551F6A95D1F7A7
:1015300083E08C930AC0220F331F441F551FFD0107
:10154000828193810197938382832030F0E03F076B
:10155000F0E04F07F0E45F0770F3FD01248335836B
:101560004683578308952F3F310581F44115510576
:101570006105710519F484E08C93089564FF03C03C
:1015800081E08C9301C01C92FD010FC02F573040A9
:10159000FD013383228383E08C9387E0440F551F42
:1015A000661F771F8A95D1F77064448355836683DD
:1015B000778308952F923F924F925F926F927F921E
:1015C0008F929F92AF92BF92CF92DF92EF92FF9253
:1015D0000F931F93CF93DF93CDB7DEB7CA1BDB0BFF
:1015E0000FB6F894DEBF0FBECDBF09942A883988A4
:1015F00048885F846E847D848C849B84AA84B984AB
:10160000C884DF80EE80FD800C811B81AA81B981B6
:10161000CE0FD11D0FB6F894DEBF0FBECDBFED01CA
:061620000895F894FFCFCD
:1016260002020202020202020000000000000000A4
:101636000001020203030303040404040404040473
:101646000505050505050505050505050505050544
:101656000606060606060606060606060606060624
:101666000606060606060606060606060606060614
:1016760007070707070707070707070707070707F4
:1016860007070707070707070707070707070707E4
:1016960007070707070707070707070707070707D4
:1016A60007070707070707070707070707070707C4
:1016B60008080808080808080808080808080808A4
:1016C6000808080808080808080808080808080894
:1016D6000808080808080808080808080808080884
:1016E6000808080808080808080808080808080874
:1016F6000808080808080808080808080808080864
:101706000808080808080808080808080808080853
:101716000808080808080808080808080808080843
:101726000808080808080808080808080808080833
:00000001FF
